:10000000A42964001720031801288A20A8010830B9
:10001000A3008B2017200318A80AAB1EA801A20C6E
:10002000A30B0928AB1AA2138B202208080038085A
:100030008400360884178004841300052B1B3606C1
:10004000FF3E0800A401A501B5129A21D33E031971
:10005000B5162D3EC63E031825280A3E031C25284A
:10006000A2000310240DA000250DA100200DA10D5C
:10007000A4070318A10A2108A507A40DA50D2208AD
:10008000A4070318A50AA90303194D289A21C63EFF
:1000900003184D280A3E03183028B51E5428A40919
:1000A000A509A40A0319A50A24089F290408A60083
:1000B00038088400F030B5050830A7000310031895
:1000C000B50A7020A60CA70B5F280000AB1A350CF0
:1000D0007020A221031470202F08A3002E080E29DF
:1000E0008413AB1F7F28000836042B1F36068000C0
:1000F000841700083604031C360680008B2800088D
:100100003604031C36062B1B36068000841736097E
:1001100080058B2835172B081F39FF3EA1002A08C0
:10012000F53E0318A10A351F1B293513A000023024
:100130004D211B29B51329080319B5170530A8004F
:100140002730A3001030B0200330A300E830B020E7
:10015000A3016430B020A3010A30B0202408B728DE
:10016000A2002508A1002408A00068212008A00002
:10017000A8030319B51329080319C1282802031875
:1001800008002008031DB513B51B0800303E9A294E
:100190000830A600A7003908840037083519800404
:1001A000FF3A351D8005F620380884003608F32014
:1001B000A001A101B518EC2038088400000836051C
:1001C000FF3EA00DA10DB51CEC20A60BDA282708D8
:1001D00035182F2920089F29390884003708800600
:1001E000000080060800841780049F29841780057A
:1001F0009F29A000A00DA00DA00D3830A005C13092
:1002000020049F000030A10032301B211F151F1950
:1002100007291E08A1001E089F29A301A200FF3084
:10022000A207031CA307031C9F290330A100DF3092
:100230001B210F29A101E83EA000A109FC30031CED
:100240002429A00703182129A0076400A10F212950
:1002500020182A29A01C2E2900002E290800A400FD
:10026000A201A3013729A10CA00CA20DA30DFF3EF2
:1002700003183329240845212208A0042308A104D7
:10028000200808000310A00DA10DFF3E031842290D
:1002900020089F290310A10CA00CFF3E03184A2937
:1002A00020089F29A20003305829A20006305829AF
:1002B000A80023082102031D5F2922082002043020
:1002C00003180130031902302805031DFF309F2950
:1002D0001030A600A501A401210DA40DA50D220832
:1002E000A4022308031C230FA50203187E29220859
:1002F000A40723080318230FA5070310A00DA10DC1
:10030000A60B6C2920089F291030A800A101A0018C
:10031000A70CA60C031C92292208A0072308031887
:10032000230FA107A10CA00CA50CA40CA80B8829D5
:1003300024089F29840031088A0030088200831332
:1003400003138312640008001630E40006118316BC
:10035000061107309F00643083120D218A15482A48
:100360000A30E700C8300D21E7030611C401C501BA
:100370000630B8000130B6000630B9000230B700D0
:10038000B5010C30C920C0002108C1000615400885
:10039000C4004108C5005C08C8005D08C9005A08CF
:1003A000DC005B08DD005808DA005908DB0056085D
:1003B000D8005708D9005408D6005508D70052086D
:1003C000D4005308D5005008D2005108D3004C087F
:1003D000D0004D08D1004608CC004708CD004408A5
:1003E000C6004508C70046084C07B2004708031876
:1003F000013E4D07B3005008B20751080318013EF3
:10040000B3075208B20753080318013EB307540854
:10041000B20755080318013EB3075608B20757083C
:100420000318013EB3075808B20759080318013EE4
:10043000B3075A08B2075B080318013EB3075C080C
:10044000B2075D080318013EB30732084807C4002D
:1004500033080318013E4907C5004408A0004508B9
:10046000A1000A30A200A3016821C4002108C50030
:100470004008A0004108A1000130A300E030552150
:100480008A11031D4C2A8A114008003CC40041080F
:10049000031C013E103CC5004408A6004508A70007
:1004A0007D30A200A3018421C4002508C5004408B2
:1004B000A0004508A1006430A200A3016821CA0081
:1004C0002108CB004008A0004108A1000130A30092
:1004D000E03052218A11031D762A8A1158304A07CA
:1004E000DE0002300318013E4B07DF004008A00089
:1004F0004108A1000130A300E03055218A11031DFD
:100500008A2A8A114A08583CDE004B08031C013E27
:10051000023CDF002C305E02C4000030031C013EB0
:100520005F02C5006408C4070318C50A4408A00098
:100530004508A1000230A300583052218A11031D42
:10054000A42A8A112D30E8004408A0004508A10023
:100550000230A300583055218A11031DB22A8A1196
:100560002B30E8004408A0004508A1000230A30099
:10057000583052218A11031DC62A8A114408583C5A
:10058000C4004508031C013E023CC5004408A0000D
:100590004508A1000230A300573055218A11031DE0
:1005A000D82A8A115830C4020230031C013EC50209
:1005B00064006708003C8A11031DE12A8A118A152C
:1005C0004B2AB229BA01BB010130F920BA00210837
:1005D000BB003A08A0003B08A1004030A200A301E4
:1005E0006821BA002108BB003A08A6003B08A70012
:1005F0000A30A200A3018421BA002508BB00923072
:10060000BA021430031C013EBB023A08A0003B08AA
:10061000A100A301003055218A11031D122B8A115C
:10062000E001E1013A08A0003B08A100A3017830F5
:1006300055218A11031D202B8A110130E000E101B0
:100640003A08A0003B08A100A301F03055218A110F
:10065000031D2E2B8A110230E000E1013A08A000B0
:100660003B08A1000130A300723055218A11031DFF
:100670003D2B8A110330E000E1013A08A0003B085D
:10068000A1000130A300EA3055218A11031D4C2B33
:100690008A110430E000E1013A08A0003B08A10003
:1006A0000230A300623055218A11031D5B2B8A1191
:1006B0000530E000E1013A08A0003B08A10002304B
:1006C000A300DA3055218A11031D6A2B8A110630E6
:1006D000E000E1013A08A0003B08A1000330A300BC
:1006E000523055218A11031D792B8A110730E00001
:1006F000E1013A08A0003B08A1000330A300D43078
:1007000055218A11031D882B8A110830E000E10170
:100710003A08A0003B08A1000430A3004C3055214A
:100720008A11031D972B8A110930E000E1013A0874
:10073000A0003B08A1000430A300C43055218A1159
:10074000031DA62B8A110A30E000E1013A08A0003F
:100750003B08A1000530A300203055218A11031D5C
:10076000B52B8A110B30E000E1013A08A0003B08EC
:10077000A1000530A3007C3055218A11031DC42B34
:100780008A110C30E000E1013A08A0003B08A1000A
:100790000530A300D83055218A11031DD32B8A11AF
:1007A0000D30E000E1013A08A0003B08A10006304E
:1007B000A300343055218A11031DE22B8A110E301B
:1007C000E000E1013A08A0003B08A1000630A300C8
:1007D000903055218A11031DF12B8A110F30E00052
:1007E000E1013A08A0003B08A1000630A300EC306C
:1007F00055218A11031D002C8A111030E000E101FF
:100800003A08A0003B08A1000730A300483055215A
:100810008A11031D0F2C8A111130E000E1013A0802
:10082000A0003B08A1000B30A3008C3055218A1199
:10083000031D1E2C8A111230E000E1013A08A000CD
:100840003B08A1000830A300003055218A11031D88
:100850002D2C8A111330E000E1013A08A0003B087A
:10086000A1000830A3005C3055218A11031D3C2CE7
:100870008A111430E000E1013A08A0003B08A10011
:100880000830A300993055218A11031D4B2C8A1181
:100890001530E000E1013A08A0003B08A100083053
:1008A000A300D63055218A11031D5A2C8A11163007
:1008B000E000E1013A08A0003B08A1000930A300D4
:1008C000133055218A11031D692C8A111730E0005D
:1008D000E1013A08A0003B08A1000930A300503014
:1008E00055218A11031D782C8A111830E000E1018E
:1008F0003A08A0003B08A1000930A3008D30552123
:100900008A11031D872C8A111930E000E1013A0891
:10091000A0003B08A1000930A300CA3055218A116C
:10092000031D962C8A111A30E000E1013A08A0005C
:100930003B08A1000A30A300073055218A11031D8E
:10094000A52C8A111B30E000E1013A08A0003B0809
:10095000A1000A30A300443055218A11031DB42C94
:100960008A111C30E000E1013A08A0003B08A10018
:100970000A30A300813055218A11031DC32C8A112E
:100980001D30E000E1013A08A0003B08A1000A3058
:10099000A300C83055218A11031DD22C8A111E30A4
:1009A000E000E1013A08A0003B08A1000B30A300E1
:1009B000063055218A11031DE12C8A111F30E000F9
:1009C000E1013A08A0003B08A1000B30A30044302D
:1009D00055218A11031DF02C8A112030E000E1011D
:1009E0003A08A0003B08A1000B30A300823055213B
:1009F0008A11031DFF2C8A112130E000E1013A0821
:100A0000A0003B08A1000B30A300C03055218A1183
:100A1000031D0E2D8A112230E000E1013A08A000EA
:100A20003B08A1000B30A300FE3055218A11031DA5
:100A30001D2D8A112330E000E1013A08A0003B0897
:100A4000A1000C30A3003C3055218A11031D2C2D30
:100A50008A112430E000E1013A08A0003B08A1001F
:100A60000C30A3007A3055218A11031D3B2D8A11C9
:100A70002530E000E1013A08A0003B08A1000C305D
:100A8000A300B83055218A11031D4A2D8A11263042
:100A9000E000E1013A08A0003B08A1000C30A300EF
:100AA000F63055218A11031D592D8A112730E00097
:100AB000E1013A08A0003B08A1000D30A30034304A
:100AC00055218A11031D682D8A112830E000E101AB
:100AD0003A08A0003B08A1000D30A3007130552159
:100AE0008A11031D772D8A112930E000E1013A08AF
:100AF000A0003B08A1000D30A300AE3055218A11A3
:100B0000031D862D8A112A30E000E1013A08A00079
:100B10003B08A1000D30A300EB3055218A11031DC5
:100B2000952D8A112B30E000E1013A08A0003B0826
:100B3000A1000E30A300283055218A11031DA42DD9
:100B40008A112C30E000E1013A08A0003B08A10026
:100B50000E30A300653055218A11031DB32D8A1173
:100B60002D30E000E1013A08A0003B08A1000E3062
:100B7000A300A23055218A11031DC22D8A112E30E7
:100B8000E000E1013A08A0003B08A1000E30A300FC
:100B9000DF3055218A11031DD12D8A112F30E0003D
:100BA000E1013A08A0003B08A1000F30A3001C306F
:100BB00055218A11031DE02D8A113030E000E1013A
:100BC0003A08A0003B08A1000F30A300593055217E
:100BD0008A11031DEF2D8A113130E000E1013A083E
:100BE000A0003B08A1000F30A300963055218A11C8
:100BF000031DFE2D8A113230E000E1013A08A00009
:100C00003B08A1000F30A300BB3055218A11031D02
:100C10000D2E8A113330E000E1013A08A0003B08B4
:100C2000A1000F30A300E03055218A11031D1C2EB6
:100C30008A113430E000E1013A08A0003B08A1002D
:100C40001030A300053055218A11031D2B2E8A1167
:100C50003530E000E1013A08A0003B08A100103067
:100C6000A3002A3055218A11031D3A2E8A113630ED
:100C7000E000E1013A08A0003B08A1001030A30009
:100C80004F3055218A11031D492E8A113730E0005B
:100C9000E1013A08A0003B08A1001030A300743025
:100CA00055218A11031D582E8A113830E000E101C8
:100CB0003A08A0003B08A1001030A300993055214C
:100CC0008A11031D672E8A113930E000E1013A08CC
:100CD000A0003B08A1001030A300BE3055218A11AE
:100CE000031D762E8A113A30E000E1013A08A00097
:100CF0003B08A1001030A300E33055218A11031DE9
:100D0000852E8A113B30E000E1013A08A0003B0843
:100D1000A1001130A300083055218A11031D942E23
:100D20008A113C30E000E1013A08A0003B08A10034
:100D30001130A3002B3055218A11031DA32E8A11D7
:100D40003D30E000E1013A08A0003B08A10011306D
:100D5000A3004E3055218A11031DB22E8A113E3058
:100D6000E000E1013A08A0003B08A1001130A30017
:100D7000713055218A11031DC12E8A113F30E000C8
:100D8000E1013A08A0003B08A1001130A300943013
:100D900055218A11031DD02E8A114030E000E10157
:100DA0003A08A0003B08A1001130A300B73055213C
:100DB0008A11031DDF2E8A114130E000E1013A085B
:100DC000A0003B08A1001130A300DA3055218A11A0
:100DD000031DEE2E8A114230E000E1013A08A00026
:100DE0003B08A1001130A300FD3055218A11031DDD
:100DF000FD2E8A114330E000E1013A08A0003B08D3
:100E0000A1001230A300203055218A11031D0C2FA0
:100E10008A114430E000E1013A08A0003B08A1003B
:100E20001230A300433055218A11031D1B2F8A1154
:100E30004530E000E1013A08A0003B08A100123073
:100E4000A300663055218A11031D2A2F8A114630CE
:100E5000E000E1013A08A0003B08A1001230A30025
:100E6000703055218A11031D412F8A113A08A000C4
:100E70003B08A1003D30A200A3016821E000210849
:100E8000E1003A08A0003B08A1001330A3002E3077
:100E900055218A11031D582F8A113A08A0003B08DA
:100EA000A1003A30A200A3016821E0002108E1007E
:100EB0003A08A0003B08A1001430A3007F30552160
:100EC0008A11031D6F2F8A113A08A0003B08A10068
:100ED0003730A200A3016821E0002108E1003A08B0
:100EE000A0003B08A1001530A300903055218A11C5
:100EF000031D862F8A113A08A0003B08A100353057
:100F0000A200A3016821E0002108E1003A08A00046
:100F10003B08A1001630A300DA3055218A11031DC9
:100F20009D2F8A113A08A0003B08A1003330A2008F
:100F3000A3016821E0002108E1003A08A0003B0875
:100F4000A1001F30A300403055218A11031DAB2F93
:100F50008A11E001E1016008E2006108E300831604
:100F600025088312E90083162408A5002308A4009D
:100F70002208A3002108A20083127F088316A10083
:100F800083127408FF006A08F4006208EA006A0825
:100F90006207B20063080318013EB3007408B20789
:100FA0000318B30A7F08B2070318B30A831621088F
:100FB0008312B2070318B30A831622088312B207FA
:100FC0000318B30A831623088312B2070318B30A5F
:100FD000831624088312B2070318B30A8316250860
:100FE0008312B2070318B30A6908B2070318B30AD9
:100FF0006B08B2070318B30A6C08B2070318B30AE8
:101000006D08B2070318B30A6E08B2070318B30AD3
:101010006F08B2070318B30A7008B2070318B30ABF
:101020007108B2070318B30A7208B2070318B30AAB
:101030007308B2070318B30A75083207E2003308D1
:101040000318013EE3006208A0006308A100143009
:10105000A200A3018A158A1168218A15E500650896
:10106000EB007308F5007208F3007108F2007008D5
:10107000F1006F08F0006E08EF006D08EE006C08DC
:10108000ED006B08EC000800BA01BB0102308A11C8
:10109000F9208A15BA002108BB003A08A0003B08D5
:1010A000A100A2010130A3008A1168218A15C200A3
:1010B0002108C300080032308A110D218A1506303C
:1010C000B8000830B6008C30AA000130AB00AE0189
:1010D000AF0176308A1157208A1565308A11572062
:1010E0008A156E308A1157208A1574308A1157205C
:1010F0008A150330A9006008A4006108A5005630D5
:10110000B000B1018A119A208A1520308A11572027
:101110008A152F308A1157208A1520308A115720BE
:101120008A15A9016508A400A5015630B000B101D7
:101130008A119A208A154B308A1157208A156D30F2
:101140008A1157208A152F308A1157208A15683046
:101150008A1157208A1520308A1157208A15743039
:101160008A1157208A1565308A1157208A156D30EB
:101170008A1157208A1570308A1157208A156530D8
:101180008A1157208A1572308A1157208A156130CA
:101190008A1157208A1574308A1157208A157530A4
:1011A0008A1157208A1572308A1157208A156530A6
:1011B0008A1157208A1520308A1157208A1568080D
:1011C0008A1157208A15A9014408A0004508A100EA
:1011D0000A30A200A3018A1168218A15B2002108F1
:1011E000B3003208A4003308A5005630B000B101A6
:1011F0008A119A208A152E308A1157208A150130BB
:10120000A9004408A4004508A5005630B000B1016B
:101210008A119A208A1520308A1157208A15483061
:101220008A1157208A1575308A1157208A156D301A
:101230008A1157208A1569308A1157208A1564301F
:101240008A1157208A1569308A1157208A157430FF
:101250008A1157208A1565308A1157208A15203047
:101260008A1157208A150230A9003E08A4003F08C1
:10127000A5005630B000B1018A119A208A1573304A
:101280008A1157208A1574308A1157208A156130C7
:101290008A1157208A1574308A1157208A156930AF
:1012A0008A1157208A1571308A1157208A15753096
:1012B0008A1157208A1565308A1157208A152030E7
:1012C0008A1157208A150530A9004208A400430856
:1012D000A5005630B000B1018A119A208A150D3050
:1012E0008A1157208A150B308A1157208A15061249
:1012F0008316061214308A1183120D218A150800F4
:101300004408BC004508BD000612831606123230A0
:101310008A1183120D218A150630B8002030B600DC
:101320005430AA004030AB008A1101208A15623C7B
:10133000031D94290330A9000130B000B1018A11C6
:1013400022208A15E70006168316061264308A11D9
:1013500083120D218A150630B8000830B6005430CB
:10136000AA004030AB00AE01AF0162308A115720B5
:101370008A150330A9006808A400A5015630B00002
:10138000B1018A119A208A150330A9004408A400EB
:101390004508A5005630B000B1018A119A208A157F
:1013A0000530A9004208A4004308A5005630B0004B
:1013B000B1018A119A208A150330A9006008A4009F
:1013C0006108A5005630B000B1018A119A208A1533
:1013D0000230A9006508A400A5015630B000B10193
:1013E0008A119A208A150230A9003E08A4003F08FD
:1013F000A5005630B000B1018A119A208A15061254
:101400008316061283120800BA01BB0100308A114C
:10141000F9208A15BA002108BB003A08A6003B084B
:10142000A7000830A200A3018A1184218A1525088B
:10143000B2002008B3003208A0003308A100023037
:101440008A114D218A15BA002108BB003A08A6006E
:101450003B08A7006430A200A3018A1184218A15E9
:10146000B2002508B3005230B2022130031C013E05
:10147000B3023208A0003308A1003930A2000130C5
:10148000A3008A1168218A15BE002108BF00080048
:101490008A11B0218A158A11E2228A1544208021FE
:0814A0000422482A6300522ACD
:02400E00653F0C
:00000001FF
